:1000000088C001C2A1C0A0C09FC09EC09DC09CC0AE
:100010009BC09AC099C098C097C096C095C094C024
:1000200093C092C091C004030904180372006100D8
:10003000700068006E00650074002E006E006500A0
:1000400074000A033100300030003000050109045B
:10005000A1010901A100850109300931150026FF20
:100060000075089502810205091901290815002566
:1000700001750195088102C0C005010904A10109AB
:1000800001A100850209300931150026FF0075081D
:10009000950281020509190129081500250175013C
:1000A00095088102C0C005010904A1010901A10050
:1000B000850309300931150026FF00750895028176
:1000C0000205091901290815002501750195088106
:1000D00002C0C005010904A1010901A100850409AC
:1000E000300931150026FF007508950281020509C7
:1000F0001901290815002501750195088102C0C064
:10010000120101010000000881179D0A030101028C
:10011000030111241FBECFE5D4E0DEBFCDBF10E048
:10012000A0E6B0E0E0E6FFE002C005900D92AC3A38
:10013000B107D9F711E0ACEAB0E001C01D92A331DC
:10014000B107E1F742D30AC75BCF85B7836085BFAC
:100150008BB780648BBF83EC8093E90008950F9385
:100160001F93CF93DF939091F90019160CF0AFC055
:100170002091F6008091F5008D3209F09EC08AE54D
:10018000809361009B3009F098C0CCE0D0E0C21BA6
:10019000D109C350DF4F8881807609F080C010926A
:1001A000E7008981882359F41092E80087EE90E0F7
:1001B0009093F8008093F70030E822E077C0853014
:1001C00021F48A818093FA0068C0863009F04AC021
:1001D0008B81813009F441C0823019F4CE0176D28E
:1001E00060C0833069F58A81882349F486E290E013
:1001F0009093F8008093F70030EC24E057C08130F2
:1002000049F48AE290E09093F8008093F70030EC94
:1002100028E14CC0823049F483E690E09093F800E6
:100220008093F70030E826E141C08330E9F582E4AD
:1002300090E09093F8008093F70030EC2CE036C00B
:10024000813249F48FEB90E09093F8008093F700AF
:1002500030EC29E02BC0823239F5CE0137D2282F7D
:1002600030EC24C0883019F48CEF90E00AC089305B
:1002700021F48A818093FC0010C08A3049F487EE13
:1002800090E09093F8008093F70030E821E00EC0F2
:100290008B3019F483EC8093E90030E806C0CE017E
:1002A00043D2282F30E802C030EC20E08F81882331
:1002B00039F48E81821728F003C030E880E001C055
:1002C000822F3093AC00809360001092F9008091EF
:1002D000610084FF49C0809160008F3F09F444C0F1
:1002E000182F893008F018E0811B809360008091FE
:1002F000AC0080FD02C00BE401C003EC8F5F809373
:10030000AC002091F7003091F80086FD05C0D901BE
:10031000912FEFEDF0E011C0AFEDB0E080E090E0A4
:1003200006C0F901E80FF91FE491ED930196181743
:10033000C1F705C08D91819391509923D9F7F901A7
:10034000E10FF11DF093F800E093F7008FED90E0DE
:10035000612F55D0183019F08FEF80936000009313
:10036000DE001C5F109361009AE080B3857031F469
:100370009150D9F71092FA001092F400DF91CF91CA
:100380001F910F9108951F93DC01162F8091620039
:1003900084FF0AC08091E90098E889278093E900EA
:1003A000912FEAEEF0E007C08AE580936200F8CF73
:1003B0008D91819391509923D9F78AEE90E0612F26
:1003C0001ED01C5F109362001F910895A82FB92FB3
:1003D0008FEF9FEF41E050EA615070F02D9138E0CF
:1003E000722F782796958795269570FF02C08427EF
:1003F00095273A95A9F7F0CF809590950895E6DF77
:100400008D939D930895CF93CFB7CF93809BFECFCD
:10041000809B09C0809B07C0809B05C0809B03C058
:10042000809B01C09EC0DF93C091F600DD27C350C2
:10043000DF4F809B02C0DF91EBCF2F930F931F9371
:1004400000B32FEF00FB20F94F933F9310B34FEF12
:10045000012700FB21F93BE031C04E7F012F10B393
:10046000216028C0102F4D7F2260000000B329C0FA
:100470004B7F2460012F000010B32BC010B3477FC7
:1004800028602AC04F7E00B320612CC04F7D10B37E
:1004900020622FC04F7B00B3206432C0422700B3DC
:1004A00049934FEF0000102710FB20F910B315708F
:1004B000A9F1297F91F2012700FB21F900B3237FE5
:1004C00089F23150F0F1102710FB22F910B3277E8A
:1004D00079F2012700FB23F92F7C81F200B310276A
:1004E00010FB24F92F7971F200C010B3012700FB33
:1004F00025F92F7359F200C000B3102710FB26F91D
:10050000223040F200C010B3012700FB27F924304D
:1005100028F64F77206810B30000F9CF3B50319593
:10052000333010E41ABFB8F0C31BD0400881033C3D
:1005300041F10B3431F11981412F1F772091F400E3
:10054000121731F4093691F10D3279F0013E69F05C
:1005500022272093FB003F914F911F910F912F91E4
:10056000DF91CF91CFBFCF9118950093FB003F91C2
:100570004F911F910F912F91DF91CAB7C6FD46CFC2
:10058000F0CF0091FB00002331F31091F90011230B
:10059000A1F53430A2F13093F9000093F5001091E9
:1005A000F6003BE0311B3093F60029C00091F900C2
:1005B00001301CF50AE547FD09C03091610034FDAA
:1005C00020C000936100CEEDD0E01FC030916200EA
:1005D00034FD17C000936200C9EED0E016C00527B5
:1005E00010E002BB1FC0052722C0052727C0052732
:1005F0002CC0052710E002BB33C04AE503C042ED22
:1006000001C0432FC4E1D0E032E011B31560909AED
:1006100002B311BB5F9355E020E820FF052702BB22
:10062000279517951C3FD8F620FF0527279502BB75
:1006300017951C3FC0F620FF05272795179502BB8D
:100640001C3F98F620FF0527279517951C3F02BBF6
:1006500070F600C0499120FF052702BB279517952A
:100660001C3F38F620FF0527279502BB17951C3F36
:1006700038F520FF05272795179502BB1C3F10F57D
:1006800020FF0527279517951C3F02BBE8F4242F70
:100690003A9519F60A7F5F9102BB00C01091FA00EB
:1006A000C651D04011F01093F40010E41ABF01605D
:1006B00011B31A7F402F4A7F02BB11BB42BB4BCF05
:1006C0000527D3CF0527D8CF0527DDCFFC018081B3
:1006D000807641F58181863029F583818230D1F0A1
:1006E000823269F08130F1F48091B1009091B200D2
:1006F0009093F8008093F7008091B3000895809163
:10070000AE009091AF009093F8008093F700809135
:10071000B000089587E790E09093F8008093F70089
:1007200082E2089580E00895DC0127EB30E0309309
:10073000F8002093F7008C918076803209F043C056
:1007400011968C911197823091F08A3001F18130AD
:10075000D1F51092B400E091B500F091B600078495
:10076000F089E02DC90112966C91099508951296B1
:100770009C91892F8150883030F5892F90E08E53DD
:100780009F4F9093F8008093F70081E008951296B0
:10079000EC911297EE2359F4E3ECF0E013968C9170
:1007A0001397819380E0EB3CF807C1F70CC08E2FC4
:1007B0008150883040F4F0E0EE53FF4F13968C9157
:1007C000808380E0089580E008958F929F92AF9299
:1007D000BF92CF92DF92EF92FF920F931F93DF931E
:1007E000CF93CDB7DEB728970FB6F894DEBF0FBE14
:1007F000CDBFFE01319688E0DF011D928A95E9F7B1
:10080000B89A87B3897F87BB88B3866088BBC09856
:1008100080E395E70197F1F786B390E086709070DA
:1008200095958795823009F4E6D0C0D2FC0190936B
:10083000B6008093B500838194819093AF0080933C
:10084000AE0081818093B00087819085009731F060
:100850009093B2008093B100858107C080E091E061
:100860009093B2008093B10069D38093B3008091DC
:10087000B0008093900014BA8FEF85BB88EF82BBE5
:1008800085E081BB11BA83BF8FE085BD84EC83BD59
:10089000E091B500F091B6000184F285E02D099554
:1008A00054DCE091B500F091B6000384F485E02DAE
:1008B0000995789490E8892E81E0C82ED12C99244E
:1008C00093945E010894A11CB11CA89548DC08B65D
:1008D00007FC02C0FF242AC088BEE091B500F09159
:1008E000B6000384F485E02D0995FF2400E010E0B4
:1008F00012C00584F685E02D802F8F5F099588232F
:1009000041F0C601002E02C0880F991F0A94E2F739
:10091000F82A0F5F1F4FE091B500F091B60080817B
:10092000992787FD9095081719071CF308B600FE54
:1009300029C098BE4091B5005091B600D50120E085
:1009400030E018C0F901ED53FF4FE081EE2379F05C
:100950008C91853018F085508C9309C0EC93C601BA
:10096000022E02C0880F991F0A94E2F7F82A2F5F1F
:100970003F4F1196FA018081992787FD909528179E
:10098000390704F3FF2009F4A0CF00E010E0EF2CBA
:10099000FF24E7FCF09422C0C701002E02C0959509
:1009A00087950A94E2F780FF17C08091620084FF68
:1009B00013C0602F6F5F0784F089E02D87EB90E014
:1009C0000995682F87EB90E0DEDC02C0C8DBA895B4
:1009D0008091620084FFFACF0F5F1F4FE091B50056
:1009E000F091B6008081992787FD90950817190727
:1009F0000CF06BCFD1CF1092AA0008958091CB005C
:100A0000882309F44DC0AC9A80E38A95F1F7AC983D
:100A100060E070E020E030E098E1892F8A95F1F7FE
:100A2000AD98660F770F9B9B61609A9B7160892FD1
:100A30008A95F1F7AD9A2F5F3F4F2830310569F75E
:100A400040E050E020E030E098E1892F8A95F1F70E
:100A5000AD98440F550F9B9B41609A9B5160892F25
:100A60008A95F1F7AD9A2F5F3F4F2830310569F72E
:100A700080E090E038E1232F2A95F1F7AD98232FFD
:100A80002A95F1F7AD9A019688309105A1F7609308
:100A9000CE007093CF004093D0005093D1000895C2
:100AA0008091CD00882309F475C0AC9A80E3982F1B
:100AB0009A95F1F7AC988A95F1F7C59A88E18A95ED
:100AC000F1F720E030E050E060E098E1AD98892F48
:100AD0008A95F1F7550F660F9B9B51609A9B616059
:100AE000AD9A892F8A95F1F72F5F3F4F2830310556
:100AF00069F75093CE006093D00020E030E098E199
:100B0000AD98892F8A95F1F7569566959B9B50680D
:100B10009A9B6068AD9A892F8A95F1F72F5F3F4FB6
:100B20002830310569F7C59888E18A95F1F720E00A
:100B300030E090E040E078E1AD98872F8A95F1F7BA
:100B4000990F440F9B9B91609A9B4160AD9A872FB0
:100B50008A95F1F72F5F3F4F2830310569F7909361
:100B6000D2004093D40020E030E078E1AD98872FA8
:100B70008A95F1F7969546959B9B90689A9B40685D
:100B8000AD9A872F8A95F1F72F5F3F4F28303105B7
:100B900069F749C0AC9A80E38A95F1F7AC9820E0F8
:100BA00030E050E060E090E040E078E1872F8A9507
:100BB000F1F7AD98550F660F990F440F9B9B51604D
:100BC0009A9B6160999B9160989B4160872F8A9561
:100BD000F1F7AD9A2F5F3F4F2830310539F7509329
:100BE000CE006093D0009093D2004093D40020E0D8
:100BF00030E078E1872F8A95F1F7AD9856956695A4
:100C0000969546959B9B50689A9B6068999B9068C7
:100C1000989B4068872F8A95F1F7AD9A2F5F3F4FD9
:100C20002830310539F78091AA00882321F180917D
:100C3000CC005F3F11F4816001C08E7F8093CC00B7
:100C40008091CC006F3F11F4826001C08D7F809352
:100C5000CC008091CC009F3F11F4846001C08B7F59
:100C60008093CC008091CC004F3F11F4886001C08C
:100C7000877F8093CC008091CC0080FD50E0509322
:100C8000CF0081FD60E06093D10082FD90E0909301
:100C9000D30083FD40E04093D50008951F931FB714
:100CA000F894A49AA59A84B3807F84BB85B38F609F
:100CB00085BBAD9AAC98BD9AC59A1092CC009EDEC9
:100CC0008091AA00882321F58091CF008F3F29F4DD
:100CD0008091CC0081608093CC008091D1008F3FC7
:100CE00029F48091CC0082608093CC008091D30065
:100CF0008F3F29F48091CC0084608093CC00809158
:100D0000D5008F3F29F48091CC0088608093CC007F
:100D1000AC9A80E38A95F1F7AC9880E090E030E0FF
:100D200040E058E1252F2A95F1F7AD989B9905C031
:100D30008331910519F441E001C03F5F252F2A95C9
:100D4000F1F7AD9A01968831910561F7442329F0B6
:100D5000373119F481E08093CB00C5989A9B10C07D
:100D6000AC9A90E3892F8A95F1F79A9909C0AC98CB
:100D7000892F8A95F1F79A9B03C081E08093CD007B
:100D8000C59A9A9B10C0AC9A90E3892F8A95F1F787
:100D90009A9909C0AC98892F8A95F1F79A9B03C05C
:100DA00081E08093CD001FBF1F9108958CE490E0F7
:100DB00090939D0080939C0089E990E00895CF93E3
:100DC000DF93EC01653010F080E094C08091CB009F
:100DD000E62FFF27E7FDF095882359F1DF011197F2
:100DE0002097F9F06883FD01E253FF4F808180FD79
:100DF00002C090E801C09FEF81FD90E09983FD0162
:100E0000E253FF4F808182FD02C090E801C09FEF56
:100E100083FD90E09A83FD01E253FF4F8081807F44
:100E20008B83FD01E253FF4F8081AA52BF4F8C9309
:100E300060C0DF011197209709F44FC06883BD019E
:100E4000660F771FFB01E253FF4F808180FD02C0D8
:100E500090E801C09FEF81FD90E09983FB01E25390
:100E6000FF4F808182FD02C090E801C09FEF83FDAB
:100E700090E09A838091CC0090E00A2E02C0959574
:100E800087950A94E2F7FB01E253FF4F80FF03C00E
:100E90008081807F21C06081462F50E09A012074BC
:100EA000307075E0359527957A95E1F7CA01807223
:100EB000907033E0959587953A95E1F7282B661F5A
:100EC0006627661F262B4071507055954795242B39
:100ED00081818295807F822B8B83FD01EE0FFF1F26
:100EE000DF01A253BF4F8D919C91EA52FF4F918336
:100EF000808384E0DF91CF91089581509091CB0061
:100F0000A82FB0E0992361F020E0FD01EA52FF4FE5
:100F1000A253BF4F9C918081981771F021E00CC0C3
:100F2000BD01660F771FCB0182539F4F6A527F4FDF
:100F300042E050E006D0282F822F089582E190E011
:100F40000895FB01DC0104C08D910190801921F40A
:100F500041505040C8F7881B990B0895F894FFCF73
:100F6000FF5A5A140334006E006500730034007396
:100F7000006E006500730009022200010100803C40
:100F80000904000001030000000921010100012201
:100F900000000705810308000A04B40000000000F7
:0C0FA00000004E06FE047D07DF06010085
:00000001FF
